:1000000000308A002F2800001F1383161F149F1032
:100010001F119F111F169F121F1383129F131F146E
:100020000030A1001F08C33921049F008316051169
:10003000831205110C3095000030A10006389200A3
:10004000FF308316920085108312851083160512E7
:1000500083120512831685128312851240288401AB
:100060001F3083051F1383161F149F141F159F1520
:10007000073083129F00603083168F00831204289C
:100080009F149F1841281E08AB01AA002A08A60742
:100090002B0803182B0FA707003003180130A807FF
:1000A000003003180130A907AE0A2E087F3C031860
:1000B0009628290CA300280CA200270CA100260CCE
:1000C000A000A30CA20CA10CA00CA30CA20CA10CD0
:1000D000A00CA30CA20CA10CA00CA30CA20CA10CB4
:1000E000A00CA30CA20CA10CA00CA30CA20CA10CA4
:1000F000A00C2008AC002108AD002C08B000013095
:100100002D07B100B10CB00CB10CB00CB10C300823
:100110009300B10C310C3039A0001508CF39200400
:100120009500A901A801A701A601AE011108AF0021
:100130002F088C3C0318A5282F08CC3C031CA528AD
:10014000203083168F00A8288312603083168F001A
:0601500083124028630049
:02400E00C430BC
:00000001FF
